:1000000083018B018A01850186018C019D018F018D
:100010009001910192019301940195019801990138
:100020009A01AB01AC01AA01831610308500FF30A4
:10003000860081176400A730810083128501860144
:1000400005110510851015309E009F019F0B262875
:100050009E0B26280F3086053030860483160F301D
:100060000605860083120515051107309E009F01C5
:100070009F0B38289E0B38280515051101309E006E
:100080009F019F0B41289E0B41280F308605203091
:100090008604051505112830E8200830E8200130D5
:1000A000E8200C30E8200630E8200730A1000321CA
:1000B000A4000830A1000321A5000B30A1000321FA
:1000C00003192A150F30A100032103197D28FB20F5
:1000D0000030A10021088900A62088000C214030B2
:1000E0008038E820B72021089520D520FB20210862
:1000F0000F3C031C7D28A10A6A280130E820061C59
:10010000392A61298207003400340A34003400346B
:10011000643400340334E8340034273410340134B8
:100120008634A0340F3442344034820730343134C2
:100130003234333434343534363437343834393473
:1001400041344234433444344534463482070D3418
:10015000BC3436340D34BB340A3400341434013426
:1001600000340034FF34FF34323405340034831655
:10017000F0300604860018308500831205108514BF
:1001800005150608F0399B00051100000000051553
:100190000511060E0F391B049B1BB728851083160B
:1001A0000F3006058600831208009600B7200F3036
:1001B00086051608F0398604851005140515051105
:1001C0000F308605160EF039860405150511080056
:1001D0009600B7200F3086051608F0398604851082
:1001E0000510051505110F308605160EF039860429
:1001F000051505110800FF309E009F019F0BFE288A
:100200009E0BFE280800831221088900831608141B
:1002100083120808A200080083168B1308155530B6
:100220008900AA3089008814881814298B170800BF
:100230002A120F089302031823299403940A031D1A
:100240002229950394031008940203182829950382
:100250001108950203182A1608002A120F0893079E
:10026000031C3829940F38290130950703182A16E2
:1002700010089407031C3D29950A110895070318D7
:100280002A16080027088F002808900029089100E6
:1002900008002A13013013020318532901301402F5
:1002A000031853292A1708000330861C0030A100C8
:1002B00003219500A10A03219400A10A03219300C0
:1002C000080000308038E820B7204530D520453080
:1002D000D5202030D5204D30D5204F30D52044308A
:1002E000D5204530D5202D30D5203130D5202E30A9
:1002F000D5203430D520FB20FB20FB2006080F3909
:10030000031D61290130E820B720A101A201A3014A
:10031000061C9129A10A21080F3C031CA101FB2006
:100320002310861C9529A20AFB20061D9929A203E9
:10033000FB20861DBA29FB2021088900220888009D
:100340000C210130E820B7202A30D5205330D520A9
:100350004130D5205630D5204530D5204430D520E9
:100360002A30D520FB20FB20FB20FB200130E82099
:10037000B720A3014130D5204430D5204430D520CA
:100380005230D5203A30D5202318C8290321231410
:100390002108F0398E000E0E9520D52021080F3946
:1003A0009520D52040308038E820B7204430D52033
:1003B0004130D5205430D5204130D5203A30D52099
:1003C0002208F0398E000E0E9520D52022080F3914
:1003D0009520D52000308038E820B72088299B015F
:1003E0000C089C00822098020318FF290130990212
:1003F0000318FF2901309A020318FF291B149C03DC
:100400001C088220990203180A2A01309A02031854
:100410000A2A1B149C031C0882209A020318122A21
:100420000314132A1B0C00349B010C089C0082202F
:100430009807031C242A01309907031C242A013041
:100440009A07031C242A1B149C031C08822099076A
:10045000031C2F2A01309A07031C2F2A1B149C030C
:100460001C0882209A07031C372A0314382A1B0C05
:10047000003411308C0009308D008E0106309D0053
:10048000EF2103184A2A8E0A8D03031D402A0330E8
:100490008C024D2A142203308C0209308D0010305A
:1004A0001D079B009B031B0884000E088E01800023
:1004B0009D0301300C07031D402A18088F00AA1E57
:1004C000632A0610861106309D0021080605A20049
:1004D000A219762A07308038E820B7202030D520AE
:1004E0000B308038E820B7202030D520003080380D
:1004F000E820B7208608A1000F301D0784000008FF
:100500000319852A3038D5208E2A06301D02031D96
:100510008C2A2030D5208E2A3030D5202A1D972ACB
:100520000C30A1000321031D992AAA179D2A8619C0
:100530009D2AAA130230A600A42A0130A6000A3080
:10054000A1000321031DAA2A26081D02031DAA2AB1
:100550002E30D5202A1DAF2AAA1BB32AB12A86190C
:10056000B32A0530B42A04301D02031DB92A2E30E7
:10057000D5200930A1000321031DC62A01301D0228
:10058000031DC62A40308038E820B7209D0B7C2A06
:100590000A30A1000321031DD32A0F301D07840058
:1005A00000083038D5202030D5204D30D5204830B7
:1005B000D5207A30D5202A1DEB2A2030D5202A1CC0
:1005C000E92A0619E62A4C30D520EB2A4630D520F8
:1005D000EB2A2030D52000308038E82097018101B7
:1005E000000000009D01C7309E000B309F000530C9
:1005F000A0008B011030850083161F308500831208
:100600000B1D052B970A0B11082B000000000000A2
:100610009E0B002BC7309E009F0B002B0B309F00C2
:10062000A00B002B0610861182308E000B1D1B2B99
:10063000970A0B111E2B0000000000008E0B162BDA
:1006400024088E008E0B222B25088E0000008E0BB6
:10065000262B030186001030850083161730850095
:1006600083120B19970A0B110108990017089A00B9
:100670009B019B0A851585110B11010819020319AD
:10068000392B9B0A9B099B0A1B0A98001030850096
:1006900083160430850083122A1DCD2B0619CD2B1D
:1006A00018089300190894001A0895008316F6306C
:1006B0000605860083122A18942B0D30A100032111
:1006C0002B02031D662BAA186F2B682BAB0ACD2BB0
:1006D0001808A7001908A8001A08A900AA1442219E
:1006E000182149212A1F7E2B0E30A10003212C0244
:1006F000031DCC2B2A14AA10AC01CD2B02308F0085
:10070000900191012A1E8E2BFD308F00FF3090004A
:10071000FF3091002D212A1A912B742B2D212A1A9A
:10072000742BAB01AA10CD2BAA124221182149210A
:100730002A1BCA2B13089B002A1AB92B06148611F0
:100740009B0A0319A52B9B0A0319AA169101900174
:100750000A308F002D212A1ACA2B0E30A100032146
:100760002C020319B52BAC0ACD2B2A10AC01AB011E
:10077000CD2B061086159B030319C02B9B03031971
:10078000AA16F6308F00FF309000FF3091002D2127
:100790002A1AAD2BAC01CD2BAC0A54210630A10096
:1007A00003210319FE2B2A19D72B0619FE2B1A0831
:1007B00091001908900018088F000519F72B1821CF
:1007C0002A1AF82B542115089B00110895001B08C4
:1007D000910014089B00100894001B089000130857
:1007E0009B000F0893001B088F001821F82B2D2168
:0E07F00015089A001408990013089800392A79
:00000001FF
